:100000000F308A004B2F0000FF00030E8301A50074
:100010007F08A4000A08AB008A01A40E0408A60009
:100020002008A7002108A8002208A9002308AA0088
:10003000831383120B1E1E288B1839288C308400E2
:10004000001C24280C183B288B1E28280B193D283F
:10005000260884002708A0002808A1002908A2007B
:100060002A08A3002B088A00250E8300FF0E7F0EAE
:1000700009008A1173288A116F288A114A280A10E8
:100080008A100A11820770346E3475346D3420344E
:100090006B340034521C53288F018E01C801C030CC
:1000A000810052106C280F08A3000E08A0000F0852
:1000B0002302031D53282008C0002308C100C90AD9
:1000C0004808073C03186C28D2144108003C031868
:1000D0006C2883160C1083120B118A112828C80A69
:1000E0000C108A1128280B1246088316BC00BC0B82
:1000F0007728831253187C28D31C8028000080287E
:10010000000042088316BC003C0883124702031813
:1001100089288316BC1C8E2800008E283C1D94283C
:100120000000000000009428000083124218A82854
:1001300000009F149F189A2883161E088312D40764
:100140001E0803181E0FD50783160117B528831242
:100150009F149F18A92883161E088312D4021E0814
:10016000031C1E0FD502831601138312C20A031942
:10017000C30AD51EBF28551EBF28CE0AD512430874
:100180000E3C031CC928031DC82842087F3C0318E5
:100190000B168B108316BC0183128B18D72883167D
:1001A000BC1ED4288312D728BC0ACC2883128B10FB
:1001B0008A11282879308400831300080319ED2858
:1001C0000630A100A001A00BE328A10BE2287B30A0
:1001D000A000A00BE928800BE02808008316321845
:1001E000F52883128713F72883168312871783163F
:1001F0008713B218FF28831207130129831683126D
:1002000007178316071332190929831287110B293F
:1002100083168312871583168711B2191329831247
:1002200087121529831683128716831687120330C7
:100230008312A000A00B1A29831686138312861737
:100240000330A000A00B2229831686138312861385
:10025000080083160613831206136330A000A00B58
:100260002F2932298316AF0803193A29061383125E
:1002700006178316300EB1000F30B1053108B200F9
:100280008312EE20831630080F39B100B2008312BA
:10029000EE200330A000A00B4B29AE08031D54290B
:1002A0008316061383120613080080308316AE00EF
:1002B00083122C0F5C296829AC0803196229831664
:1002C0002E1783128316AF012E08B0008312292146
:1002D0002F088316AD002D08831203178D00831697
:1002E0008C130C1483120C0883160313AC002C0F10
:1002F0007A29902983122D088316AC0683122F08C1
:100300008316AF002C08B00083122921AD08031911
:100310008D2983162C088312AD008316AD0A6B2934
:1003200083122F0883162D02031DA229AD012D1A59
:10033000A2290130AF002030B0008312292183169A
:10034000AD0A972983122D08493C0319AD01080015
:100350000830F300FA30F900DA20F30BAA2908007C
:100360006430F900DA2008005521B021AE08031DE1
:10037000AE0308006D08FD006C08FC006B08FB0074
:100380006A08FA008316A301A2017908A10078087F
:10039000A0002030A800A401A501A601A7017D08A6
:1003A0008312A3007C08A2007B08A1007A08A000A9
:1003B0000310201CEB2983162008A407210803182A
:1003C000210FA50722080318220FA60723080318E8
:1003D000230FA70783128316A70CA60CA50CA40C49
:1003E0008312A30CA20CA10CA00C8316A80BF92954
:1003F000FB298312D82983122308ED002208EC0080
:100400002108EB002008EA000800B630A000A30194
:10041000A201A1017708780479047A04031D122A45
:10042000A0011F2A0310A11B1E2AF70DF80DF90DBC
:10043000FA0DA30DA20DA10DA00B122AA113080005
:100440007808EA027908031C790FEB020030031CDC
:100450000130EC020030031C0130ED020800770887
:100460000319122B8316A4007B08031D392A83125B
:10047000122BA402031C432A7F30A407031C422A28
:100480008312122B4D2A8130A4020318492A8312A9
:10049000122B031D4D2A8312122B24088312A00055
:1004A000A101A201A3018316A3017808A200A2174B
:1004B0007908A1007A08A0001930A4007E08A002E3
:1004C0000318722A0130A1020318722AA20203182B
:1004D000722AA3020318722AA30AA20AA10A7E089A
:1004E000A007A62A7D08A10203188D2A0130A202C6
:1004F00003188D2AA30203188D2AA30AA20A7D08D5
:10050000A1077E08A007031CA62AA10A031DA62A8C
:10051000A20A031DA62AA30AA62A7C088038A202E2
:100520000318A32A0130A3020318A32AA30A7C08F4
:100530008038A2077D08A107031C812AA20A031D97
:10054000812AA30A812A831223148316A40BA92AC1
:10055000B62A0310A00DA10DA20DA30D0310831246
:10056000A30DA20DA10D8316A50D5E2A251CC02A80
:1005700003108312A10CA20CA30C8316A50CC52A90
:100580008312A0030319122B8316A51BEE2A031056
:10059000A00DA10DA20DA30D7E08A0020318DA2A5A
:1005A0000130A1020318DA2AA2020318DA2AA302F0
:1005B000031C052B7D08A1020318E52A0130A202C5
:1005C0000318E52AA302031C052B7C088038A2022D
:1005D0000318EE2A0130A302031C052B8312A30A81
:1005E0000319F42A8316052BA20A0319F92A831684
:1005F000052BA10A0319FE2A8316052BA00A03194D
:10060000122BA10CA20CA30C83167808A4007C0862
:10061000A406A41F0F2B8312A117162B8316831277
:10062000A113162BA001A101A201A30108007708C4
:100630000319AE2B8316A0007B08031D212B831208
:10064000AE2BA00703182F2B7F30A00203182A2BF4
:100650008312AE2B031D2E2B8312AE2B352B813034
:10066000A007031C352B8312AE2B20088312A00099
:10067000A101A201A30178088316A400A417790898
:10068000A3007A08A2001830A000A101221C6B2B45
:100690007E088312A307031C562BA20A031D562BA8
:1006A000A10A031D562B8316A11783127D08A207EA
:1006B000031C602BA10A031D602B8316A117831254
:1006C0007C08F900F9177908A107031C6A2B831627
:1006D000A11783128316A10D8312A10CA20CA30CE7
:1006E0008316A40CA30CA20C0310A00B452B013005
:1006F0008312A0070318AE2BA11B872B8316A40D12
:100700008312A30DA20DA10DA0030319AE2B831616
:10071000A41FA12B8312A30A0319902B8316A12BCC
:10072000A20A0319952B8316A12BA10A03199A2B50
:100730008316A12BA10CA20CA30CA00A0319AE2BAB
:1007400083167808A1007C08A106A11FAB2B831299
:10075000A117B22B83168312A113B22BA001A10102
:10076000A201A301080080308318FC068316A201B1
:10077000A3017808A1007C08A10677080319BB2C07
:10078000A0008312A0007B080319C72C8316A002C7
:100790000319552C031C0D2C7C08A600A6177D08F8
:1007A000A5007E08A400A3010310A60CA50CA40CB0
:1007B000A30CA00BD32BA11FE02B2214E22C2210A0
:1007C000201022167A3084008313F72C2212A11BEA
:1007D000F52B201C022CA60CA50CA40CA30C831238
:1007E000A00A0319DC2C8316022CA61B052C03106F
:1007F000A30DA40DA50DA60D8312A0030319DC2CD7
:100800008316F52B2217772C22137808A100A11F3D
:100810000B2CA617D02CA613D02C7B08A00083127B
:10082000A00077088316A0027808A600A61779080A
:10083000A5007A08A400A3010310A60CA50CA40C23
:10084000A30CA00B1B2CA11F282CA214E22CA2107D
:100850002010A2167E3084008313F72CA212A11B55
:100860003D2C201C4A2CA60CA50CA40CA30C831216
:10087000A00A0319DC2C83164A2CA61B4D2C03104E
:10088000A30DA40DA50DA60D8312A0030319DC2C46
:1008900083163D2CA217772CA2137C08A100A11F60
:1008A000532CA617D02CA613D02C7C08A600A61774
:1008B0007D08A5007E08A400A11F622CA6132215A6
:1008C000E22C2211A30120107A3084008313F72C2C
:1008D000A11B8F2C7808A100201C772CA60CA50C3E
:1008E000A40CA30C8312A00A0319DC2C8316A31FEB
:1008F0008A2CA40A031D8A2CA50A031D8A2CA60A89
:10090000031D8A2CA60CA50CA40C8312A00A0319A3
:10091000DC2C8316221B042CA21B4C2CB52C803003
:10092000A606A61F972CE22C7C08A100A62C78080E
:10093000A100A608031DA62CA508031DA62CA4082B
:10094000031DA62C8312A0018316D02CA61BB52C48
:100950000310A30DA40DA50DA60D8312A00BB12CA1
:10096000B32C8316A62CDC2C8316A11FB92CA6173A
:10097000D02CA613D02C7B088312A0007C088316F1
:10098000A6007D08A5007E08A400D02C831277085D
:10099000A00078088316A6007908A5007A08A400AC
:1009A00026088312A100831625088312A20083164D
:1009B00024088312A300162DA001A101A201A30106
:1009C000162D8316A301A409A509A609A309A30A44
:1009D000031DF02CA40A031DF02CA50A0319A60A76
:1009E0002218DF2BA218272C2219612C942C000826
:1009F000A407031C012DA50A031D012DA60A031936
:100A0000201484030008A507031C092DA60A031956
:100A1000201484030008801F803AA60703182014BE
:100A2000221AE62BA21A2E2C682C831208006D08BD
:100A30008316B10083126C088316B00083126B0812
:100A40008316AF0083126A088316AE00B501B401A5
:100A50002D08B3002C08B2008312A001A101A2014D
:100A6000A3018316B601B701B801B90135083404F2
:100A70003304320403196E2D2030BA000310AE0D7A
:100A8000AF0DB00DB10DB60DB70DB80DB90D3508E0
:100A90003902031D552D34083802031D552D330826
:100AA0003702031D552D32083602031C662D32080D
:100AB000B6023308031C330FB7023408031C340F8B
:100AC000B8023508031C350FB90203148312A00DB8
:100AD000A10DA20DA30D8316BA0B3E2DB6308400D6
:100AE000831383122308ED002208EC002108EB0099
:100AF0002008EA0008007708B63CF700A301780850
:100B0000FB00F8170310F80CF90CFA0CA30CA20C5C
:100B1000A10CA00CF70B822DFB1F992DA009A10998
:100B2000A209A309A00A0319A10A0319A20A031919
:100B3000A30A0800B021F101F001EF01EE01521407
:100B4000D210C501C401FF30C900C801FE308100C8
:100B50008F018E010B1183160C1483128B16C0307B
:100B60008B043230F900DA205218C32D521EBD2DED
:100B7000D218BC2DC81FB82DC32DD218C32D4808BC
:100B8000273C0318BD2D0B138B138B1BC42D8B120D
:100B900083160C108312D21CBF2EF4014908F300F7
:100BA000F30DF40DF30DF40DFC30F305F30A031906
:100BB000F40AED013030EC00D430EB00EA017408A7
:100BC000F9007308F800BA216D08FA006C08F90002
:100BD0006B08F8006A08F70005222308F1002208D4
:100BE000F0002108EF002008EE00ED014808EC00BD
:100BF0004008EA004108EB00F9013630F8002022F5
:100C00006D08FA006C08F9006B08F8006A08F70034
:100C100005227108FA007008F9006F08F8006E08E4
:100C2000F7002308FE002208FD002108FC00200830
:100C3000FB002F222308F1002208F0002108EF001A
:100C40002008EE007108F8007008F7006F08F60041
:100C50006E08F5008E30A0007508A0027608A2008C
:100C60007708A100A217A0080319412E0310A208BB
:100C7000031D3D2EA1080319412EA20CA10CA00BAF
:100C8000362EF61F482EA109A209A10A0319A20AAD
:100C90002208C5002108C4007108FA007008F90094
:100CA0006F08F8006E08F7007108FE007008FD007C
:100CB0006F08FC006E08FB0017232308F1002208D0
:100CC000F0002108EF002008EE00521E812E831054
:100CD0007108FA007008F9006F08F8006E08F70054
:100CE0009A30FE009930FD001930FC007E30FB0088
:100CF000B3232308F1002208F0002108EF002008A8
:100D0000EE00F9010730F800BA2174088316AD002F
:100D10007308AC00831217256B08C7004430C70264
:100D20005310D3100130C6004708023C03189C2E14
:100D30000330C702C60A942E47185314C718D31499
:100D40006A08C700F830C7057108FA007008F90092
:100D50006F08F8006E08F7007B252308ED002208D5
:100D6000EC002108EB002008EA008316AD013730C3
:100D7000AC00831217256B08D5006A08D400080060
:100D8000EA09EB09EC09ED09EA0A0319EB0A031970
:100D9000EC0A0319ED0A08000730F300203083162F
:100DA000A000A100A200A300A400A500A6003F305F
:100DB000A7002030A800A900AA00AB018312531D90
:100DC000E62E3D308316A200E92E83123D308316B5
:100DD000A10083124B081E3C031DF52ED21CF52EDC
:100DE0008316A0010130A10083125312ED1FFA2EC9
:100DF0005316C026AC08031D582F6D08FA006C0866
:100E0000F9006B08F8006A08F700F40152190A2F7C
:100E10000430F400FA08031D1B2FF908031D1B2FD3
:100E2000F808031D1B2F7708103C031C1B2F7408A8
:100E3000063C031C222F0310FA0CF90CF80CF70CDB
:100E4000F40A0A2F0730F402F40E7708F407D218D8
:100E50002B2FFF30F4000230CF077408CF02AE080A
:100E600003193C2F4030D306531B382F8030D30654
:100E7000531F3C2FD31BAE034F08043C0318562FBF
:100E80002E085002CF00CF0CCF0C3F30CF05CF083B
:100E90000319512F0310CF0C500F4F2F502FD00A92
:100EA000472FAE080319562F5008AE007408CF0024
:100EB000D21CD82FED08031D6B2FEC08031D6B2FE0
:100EC0006B08263C0318732FFF3A031D6B2F6A082B
:100ED0000F3C0318732F8316AD010A30AC00831248
:100EE0001725CA0A5A2FF4014A08023C03187C2F1E
:100EF0000330CA02F40A742F0430CA075319CA0A0D
:100F00004A08073C0319CA0173084A02031D902FBF
:100F10007308F303A03E840083132E308000CA01BF
:100F2000F601F501EB08031D992F6A08093C031827
:100F3000A32F0A30EA020030031C0130EB02F50A4D
:100F40000319F60A922F7308F303A03E840083135B
:100F500030306A078000531DB02F0730F300531163
:100F60007608EB007508EA006A086B04031D842FFD
:100F7000CA08031D842F7308073C0319F303531E8B
:100F8000C72FA0307307840083132D3080007408AE
:100F90003F20A1008316A9008312CD080319D82F82
:100FA0004E088316A00083124D088316A1008312F9
:100FB00051088316AA008312CD014B08AF005521BA
:100FC000F30173080A3C031CF42FA030730784005C
:100FD00083130008FB0001308316AF007B08B000CC
:100FE00083122921F30AE12F08000230F800FA30B9
:0A0FF000F900DA20F80BF72F0800D3
:1010000083168612831286168A11F5278A158A118D
:101010009A258A1583168612831286120800710893
:10102000B7007008B6006F08B5006E08B40008007D
:101030003308FA003208F9003108F8003008F700E8
:101040003708FE003608FD003508FC003408FB00B8
:101050008A112F228A152008F3002108F4002208A3
:10106000F5002308F60083142308FA002208F9008B
:101070002108F8002008F700FE01FD01FC017F3087
:10108000FB008A11B3238A15080018202008F300FA
:101090002108F4002208F5002308F6003F08FA00B2
:1010A0003E08F9003D08F8003C08F7008A110522C7
:1010B0008A152308FA002208F9002108F800200800
:1010C000F7007608FE007508FD007408FC00730840
:1010D000FB008A112F228A152308FA002208F90042
:1010E0002108F8002008F7008A117B258A152308BB
:1010F000BF002208BE002108BD002008BC00080077
:10110000521E8B28B130F6006030F5006630F400D6
:10111000AE30F30093286F30F600FC30F5000F304E
:10112000F400B230F3003F08FA003E08F9003D0831
:10113000F8003C08F7008A1105228A152308FA00F6
:101140002208F9002108F8002008F7003708FE00FF
:101150003608FD003508FC003408FB008A1117230F
:101160008A157608FA007508F9007408F800730803
:10117000F7002308FE002208FD002108FC002008DB
:10118000FB008A112F228A152308FA002208F90091
:101190002108F8002008F7008A117B258A1523080A
:1011A000ED002208EC002108EB002008EA0008000E
:1011B0003308D9003208D8003108D7003008D600EB
:1011C0007108B3007008B2006F08B1006E08B0007B
:1011D00000200F20BF01BE016908BD006808BC00E7
:1011E00045203308B7003208B6003108B500300892
:1011F000B400851C0F293F08FA003E08F9003D089D
:10120000F8003C08F7008A1105228A152308BB0064
:101210002208BA002108B9002008B8001729590887
:10122000B3005808B2005708B1005608B00080203B
:10123000851829296B08DB006A08DA005A080319A7
:10124000DB03DA033D08DD003C08DC00DC0A03199F
:10125000DD0A0800F8012330A000A00B2D29D701DA
:101260000330D6009F149F18332983161E0883125B
:10127000D6071E0803181E0FD707F80A7808303C57
:1012800003183229F830D60508005930AF008A110A
:1012900055218A15080003171F109F101F119F1159
:1012A00003131F13703003179E00831603131F12BE
:1012B0009F161F1383129F171F14FF30831685007C
:1012C00007308600870003309500811383120317CF
:1012D000950199019A0183169E0183129B010313C4
:1012E0008D1203179901A1309A0083169E01831273
:1012F0009B0103138D1283160108C739283881001A
:101300000530831290000030A10092000030831657
:101310009200831294128316871306160613013067
:101320008312940000308316940018308312A100B9
:101330001F08C33921049F00831686128312861268
:1013400083160612831206128316061383120613DF
:1013500083168613831286130F30F9008A11DA2060
:101360008A15F3017319C22903308316B2008A115A
:101370008312EE208A150530F9008A11DA208A15C9
:10138000F30AB22902308316B2008A118312EE20CA
:101390008A15AF018A1155218A150A30F9008A1180
:1013A000DA208A15FF30AC008316AF014030B00060
:1013B0008A11831229218A15A630AF008A1155217E
:1013C0008A158316061671308312AD00AC01953074
:1013D000AF008A1155218A158A11A8218A1540303B
:1013E000D000FF30AE00051CFB295A30AF008A1137
:1013F000B4218A15F3298518032A6B30AF008A11AE
:10140000B4218A15FB294030AE00F20172080F3C6E
:10141000031C1D2A5A30720784008313F0307207B0
:10142000F500750803178D0083168C130C148312B6
:101430000C088000F20A0313062A8A119A258A15DD
:10144000ED01EC014508EB004408EA002A30CB002E
:101450002030D1001130CA005311CD018A11CC26A1
:101460008A15D8204508EB004408EA00AC0A113080
:10147000CA003030CB008A11CC268A158A11A821E7
:101480008A151430A1001F08C33921049F002A21A6
:101490005708C3005608C2008316861283128616A8
:1014A0000A30F9008A11DA208A152A218316861259
:1014B000831286121830A1001F08C33921049F002F
:1014C00043085702031C712A031D6A2A5608420268
:1014D0000318712A4208D6024308031C430FD7029F
:1014E000732AD701D601D708031D7A2A56087F3CF4
:1014F0000318892AAC014521E730AF008A11552134
:101500008A15AC0A45218A11A8218A158A11A821B9
:101510008A158A15632FC301C201D5010F30D4008B
:10152000CD01CE01D2104908183C0318D12A490830
:101530002B3C031CD12A1030A1001F08C339210401
:101540009F008316011383120B16C0308B04643086
:10155000F9008A11DA208A150B138B138B1BAD2A25
:101560000B121830A1001F08C33921049F00D50CAD
:10157000D40CD50CD40CD50CD40CD50CD40CD50C67
:10158000D40C0730D505CE080319CA2A0130D50777
:10159000CE03C32AD508031DD02A54081E3C031CC1
:1015A000D2140800831606128312061252168A11EC
:1015B0009A258A150800831606168312521208000F
:1015C0003308D9003208D8003108D7003008D600D7
:1015D000D211D2224408CE004508003C0318F22A5A
:1015E000FF30CE00CE080319CE0AD21CCE01DB227A
:1015F0008A119A258A15450CA300440CA200A30C5D
:10160000A20CA30CA20C2208CD004508073C03182D
:101610000B2BFF30CD00CD080319CD0AD21CCD0114
:10162000CE0803192A2B4E083B3C031C2A2B4E08DC
:10163000173C03181F2B4D084E0203182A2B4E0887
:10164000073C031C272B4D08103C031C2A2BD222DD
:10165000CD01D2140F20CD080319302BD214CE01A6
:101660004E08073C031C3B2B4D087F3C031C4D2BB5
:10167000CD0803194D2B3708B3003608B2003508E2
:10168000B1003408B00000200F20BF01BE0169087E
:10169000BD006808BC004520D2155908B3005808A1
:1016A000B2005708B1005608B000CD010800013063
:1016B000AC004521AC018A11B0218A15D21C652CE1
:1016C000051C652C8519902B05186D2B69082E3C7F
:1016D000031C6D2BE80A0319E90A8518772B6908A2
:1016E000223C0318772B68080319E903E803463006
:1016F000D100A201A3012308ED002208EC00690833
:10170000EB006808EA002430CB000230CA00500821
:10171000AE008A11CC268A158A11B0218A15622B57
:1017200083160612831206163A30A000A00B962BE1
:101730002A2157081B3C0318C42BED012330EC0071
:10174000F330EB000130EA0057088316AD00831236
:1017500056088316AC008A11831217258A15F901E1
:101760003030F8008A1120228A156A086202031DAF
:10177000BD2B6B0863020319C42B6B08E3006A08D6
:10178000E200E20A0319E30A831606160730831201
:10179000D1000F30CA00ED01EC016308EB006208D4
:1017A000EA005430CB0053118A11CC268A158A11D5
:1017B000A8218A155A30AF008A1155218A15FF30A9
:1017C000AE00051CE92B5A30AF008A11B4218A15EE
:1017D000E12B5008AE008A11A8218A158A119A259A
:1017E0008A1549082B3C0318032CD8205211452197
:1017F000851CFD2B9030AF00FF2B8B30AF008A1182
:1018000055218A15392C5508DF005408DE008B223B
:101810005508E1005408E000E0223F08E7003E08D8
:10182000E6003D08E5003C08E4005630D1000B30EE
:10183000CA004830CB005311ED01EC016108EB0008
:101840006008EA008A11CC268A158A11A8218A1517
:101850000130AC002030D1001130CA00ED01EC01A4
:101860004508EB004408EA004E30CB008A11CC2634
:101870008A15F20172080F3C031C642CF0307207C9
:10188000F3005A307207840083130008F4007308D1
:1018900003178D0074088C0083168C130C158312AB
:1018A00003130B08A0008B138316031755308D000C
:1018B000AA308D008C148C185B2C0C11831203132E
:1018C00020088B04F20A3A2C6A2C7C30AF008A1173
:1018D00055218A158A11A8218A158A157E2FA10102
:1018E000A201A001A3017B08031D792C7A0803192A
:1018F000932C1030FC000310F80DF90DA00DA30D72
:101900007B082302031D862C7A082002031C8F2CDF
:101910007A08A002031CA3037B08A3020314A10DF1
:10192000A20DFC0B7B2C0800C301C201D21BCE2DE3
:10193000521BCE2D1830CB00521183160612831283
:1019400006128A11F5278A158316061683122A2194
:101950005708F3005608F200F31BAB2D1030720746
:10196000F4007308F500273003182830F5077508D0
:10197000F9007408F800FB013130FA006F242208E6
:10198000F5002108F4008316061283120616C20A17
:101990000319C30A9F149F18CB2C83161E08F60048
:1019A00083121E08F700431BDF2C77087502031C07
:1019B000DF2C031DC72C74087602031CC72C83166A
:1019C000061683122A215708F5005608F4007208FB
:1019D000F60001307307F700431FF82C75087702F3
:1019E000031CF82C031DF72C76087402031CD21775
:1019F000C308031DFF2C4208023C0318AB2D5215EF
:101A000053150630CA004630D1007508F700740837
:101A1000F6008A11B0218A152A215608F6025708C5
:101A2000031C570FF702F70CF60CF70CF60CF70C2B
:101A3000F60CF70CF60C0F30F705CE01F719362D22
:101A4000F708031D272D7608633C03182A2DF7019C
:101A50006330F600521D2F2D7608CD00362D760806
:101A6000CE004E0B342DCE010310CE0D0430D20625
:101A70005708F7005608F600521D092D4E084D0272
:101A80000318442D3630CB003030CE004D08093CD1
:101A900003184E2D0A30CD02CE0A462D3030CD0728
:101AA0004E08303C031D582D4D08CE002030CD008F
:101AB0007208F4027308031C730FF502ED01EC01C8
:101AC000C330EB00CF30EA007308F9007208F80069
:101AD0008A1120228A155B30F9006830F8008A11DB
:101AE000BA218A1575088316AD007408AC008A11F6
:101AF000831217258A153030F900D430F8008A1186
:101B000020228A1563088316AD00831262088316AB
:101B1000AC008A11831217258A154308F900420880
:101B2000F8008A11BA218A15F9013130F8008A11BA
:101B300020228A15ED08031DAB2DEC08031DAB2DEB
:101B40006B08033C031CAB2DF9010A30F8008A1125
:101B5000BA218A15CA0383160612831206120530AB
:101B6000F9008A11DA208A152A21831606168312B3
:101B7000431FCD2D7308003C031CCD2D7508003C80
:101B80000318CD2D5708003C031CCD2DD21ECB2DA4
:101B9000D212D210CD2DD2135217D12D8A11F52782
:101BA0008A158A15852F18202008F2002108F300D5
:101BB0002208F4002308F500FA002208F9002108A1
:101BC000F8002008F7003B08FE003A08FD0039083D
:101BD000FC003808FB008A1117238A152308FA0035
:101BE0002208F9002108F8002008F7008A117B2557
:101BF0008A152308ED002208EC002108EB002008DC
:101C0000EA000630CB000230CA004630D1008A1507
:101C1000872F4830D1000730CA001230CB00D21EC7
:101C2000142ED218D212E022D219272E521E212EA3
:101C30006708BF006608BE006508BD006408BC00F8
:101C4000272EBF01BE015D08BD005C08BC008020DE
:101C5000D21D2C2E4230CB00521A402E8A11F5276D
:101C60008A155A08EA025B08031C5B0FEB0200307E
:101C7000031C0130EC020030031C0130ED02422E47
:101C8000CA0A53158A15892F53125315ED01EC0119
:101C90006108EB006008EA005F085502031C622E31
:101CA000031D562E54085E020318622E5508F900D3
:101CB0005408F8008A11BA218A155F08D5005E0819
:101CC000D400692E5F08F9005E08F8008A11BA2175
:101CD0008A1555088316AD00831254088316AC008C
:101CE0008A11831217258A155508F3005408F2004B
:101CF0004308F5004208F4008B227508C3007408FD
:101D0000C200D21C492F6B08F5006A08F400ED01EF
:101D1000EC015B08EB005A08EA005B08F9005A087E
:101D2000F8008A11BA218A156C08EA006D08EB00E8
:101D3000EC01ED017308F9007208F8008A11BA216C
:101D40008A1575088316AD007408AC008A118312D9
:101D500017258A1554087402F2007508F300550817
:101D6000031C550FF30275085502031CC72E031DF3
:101D7000BD2E540874020318C72E5316740854025B
:101D8000F2005508F3007508031C750FF302730881
:101D9000F9007208F8008A11BA218A15521FF72E2D
:101DA0006D08F3006C08F2007308F9007208F8007F
:101DB000FB010330FA006F242208F3002108F2002F
:101DC00055087302031CEA2E031DE92E5408720203
:101DD0000318D2107208D4027308031C730FD502C3
:101DE000D508031DF72E54081D3C0318D2105508C2
:101DF0008316AD00831254088316AC008A11831237
:101E000017258A15531E082F8A11C0268A15492FB7
:101E1000D21B492F521B492F42144308F900420894
:101E2000F8008A11BA218A158316AF014830B00034
:101E30008A11831229218A15CE01ED080319222F58
:101E40001F30CE00FF30CD00CD0803193E2F031008
:101E5000CD0C6C084D020318322F0310CE0DCE0AA4
:101E60001F30CE0501308316AF0083124E08831653
:101E7000B0008A11831229218A15242F4308831662
:101E8000AD00831242088316AC008A118312172515
:101E90008A158A15952F840183131F308305AD01A0
:101EA00003171F109F101F119F1103131F130030E2
:101EB00003179E0099019A0183169E0183129B01CC
:101EC00003138D124B298A119A258A150F20CC0AEB
:101ED0006F08CC024C08023C031C722FD319D21697
:101EE000D311732FD3156F08CC0049082B3C03186E
:101EF0007C2FD213521352110518572B851C882F93
:101F0000521E832FDB22D211942C521DD32D892FE8
:101F1000092EAC01D21B912F521B912F8A11CC2676
:101F20008A15AC0A521DA92F442E0730D1000B3060
:101F3000CA001E30CB00D21FA02F3C30CB00AC011A
:101F4000521FA52F8530CB00AC018A11CC268A15F3
:101F5000E52F4630D1000230CA00D21DE42F0C30EC
:101F6000CB003F08ED003E08EC003D08EB003C08CC
:101F7000EA00521ED52F53156408EA026508031CB7
:101F8000650FEB026608031C660FEC026708031C72
:101F9000670FED02ED08031DD42FEC08031DD42FAD
:101FA0006B083F3C0318D211DC2F5D08F9005C0878
:101FB000F8008A1120228A15ED1BD211D21DE32FC1
:101FC0008A11CC268A15E52FAC01AC08031DEA2F37
:081FD000AC0A4521632F6300F8
:10420000280008000C0001000600FF002000050047
:10421000200043007800FF00200020002000430021
:104220007000FF002000060020004C007800FF0016
:1042300003002000430020006D00FF000400200068
:10424000450053005200FF0020004300630061005E
:104250006C00FF0020004600300020002000FF001E
:1042600020004600430061006C00FF000300430093
:10427000200073007A00FF0020000400200052009C
:104280007800FF000500060020004C007800FF00C9
:1042900055006500730072003000FF0046006500A5
:1042A000730072002000FF00200020002000520058
:1042B0006500FF0053007700690074006300680028
:1042C000200074006F0020004D0065006100730045
:1042D0002E002100FF0020004C0078002000740018
:1042E0006F0020004300780020006D006F00640024
:1042F000650021002000FF002000450072007200D0
:104300006F00720021002000FF0002002D00450018
:1043100053005200FF004C002D003E003000FF0013
:1043200043002D003E003000FF003D000F000E0056
:104330007E001E005B004700300021007000250059
:1043400011000D000A0010003A00FF0000000000FC
:104350000300040002000500090006001800080020
:1043600018000B001A000300010003000000000009
:1043700013001400140014001300000004001F00B8
:1043800011001F0000001F000400000004000E00C8
:104390000A000A000A000E000400000004000400E5
:1043A0001F0000001F0004000400000008001D00A2
:1043B0001D001D001D001D000800000000000E0073
:1043C0001100110011000A001B000000FF004C004A
:1043D0006F00770020006200610074007400FF002D
:1043E0003E00260047002A00C70035008600100066
:1043F000FA00000093000C000500000024002700D4
:02400E00C23FAF
:00000001FF
